:020000040000FA
:020000000428D2
:08000800FF30A200FF30A3004D
:10001000BE01A01007309F00A410A5272214BA2704
:10002000A210B9272211B827A211B7272212B6278A
:10003000A212B5272314B427A315B1272316B0277E
:10004000A316AF272317AE27A317AD274030952659
:10005000A513A027A313AD270230C400A313AD2717
:1000600001308727A317AD2701308727C40B2E281F
:100070007326201E3C283E281B27382871267F39EE
:10008000A60026087A27A7002708463C031C4B2811
:100090002708A8009D282708473C031D5128A620B3
:1000A0009D282708483C031D58282708A8009D289C
:1000B0002708493C031D5E28A7239D2827084A3CA2
:1000C000031D642809219D2827084C3C031D6A282C
:1000D00039219D2827084D3C031D702809219D28A2
:1000E00027084E3C031D77282908A8009D282708CB
:1000F000503C031D7D28CF209D282708523C031D1E
:100100008328E1229D282708543C031D8928BA2012
:100110009D282708563C031D8F28AB209D282708C3
:10012000573C031D952839219D282708583C031D5D
:100130009B28B5239D283F30A8000130362727088B
:100140007127BD0028087D263828A528AC26A426BE
:100150002708A80008002708A8002030AA0031308E
:10016000AB002E30AC003130AD003030AE0020306E
:10017000AF0008002708A8002030AA005730AB00C5
:100180006930AC007330AD007030AE003630AF0077
:100190003230B0003830B1002030B20008003D08E5
:1001A000043C031D012927087D268C26201ED92802
:1001B000DB281B27D528BC08031DE12881309526A4
:1001C000FF283C08013C031DE82840309526FF2805
:1001D0003C08023C031DEF2820309526FF283C08F0
:1001E000033C031DF62815309526FF283C08043CE7
:1001F000031DFD280A309526FF283F30A800082956
:1002000004293F30A80008292317AE274030952E37
:1002100008002708A8000A303E02031825293A0ED4
:10022000F0393B074202031D22293C0EF0393D07FD
:100230004102031D2229380EF03939074302031DFC
:1002400022292429A7230F2938290A303E02031C1A
:100250003629380EF0393907C5003A0EF0393B0718
:10026000C6003C0EF0393D07BC2538293F30A800B8
:1002700008002708A8003E08013C031D4829023059
:10028000C4000430C5000830C60000309222912A14
:100290003E08023C031D55290330C4000530C5004B
:1002A0000830C60000309222912A3E08033C031D0C
:1002B00062290230C4000430C5000830C6000E3088
:1002C0009222912A3E08043C031D69293F30A80070
:1002D000912A3E08053C031D76290230C4000430F3
:1002E000C5001830C60017309222912A3E08063CFD
:1002F000031D83290330C4000530C5001830C60033
:1003000017309222912A3E08073C03198B293E0898
:10031000083C031DDE290430C4004408003C031CD3
:100320009229CC2901304402C40002302C26CB0192
:10033000013058263108CB00043058263008CB0055
:10034000043058262F08CB00043058262E08CB0046
:1003500002305826CB01013058264408003C0318CF
:10036000B32906302C263208AE003608B2003A080F
:10037000B6003308AF003708B3003B08B7003408B5
:10038000B0003808B4003C08B8003508B10039089E
:10039000B5003D08B9008D2918302C263F08EE26FF
:1003A0003E08073C031DD72917302C26D9290A30CF
:1003B0002C2606302C260430C425912A3E080A3CFF
:1003C000031D0F2AD8250D30C800300EF039310733
:1003D000C9002E0EF0392F0710260D30C800340E3C
:1003E000F0393507C900320EF039330710260D30C9
:1003F000C800380EF0393907C900360EF039370712
:1004000010260F30C8003C0EF0393D07C9003A0EE7
:10041000F0393B071026F6250830C425912A3E08FE
:100420000B3C0319172A3E080D3C031D7C2AC8010A
:100430000E30C90041081026C8016E30C900A9302D
:100440001026C8010E30C90042081026C8016E30BF
:10045000C900AA301026C8010E30C9003C0EF03980
:100460003D071026C8016E30C900A8301026C8010B
:100470008430C900A63010263E080B3C031D542AC8
:10048000C8010E30C90055301026C8016E30C900B1
:10049000A7301026C8010E30C900AA301026C801A6
:1004A0006E30C900A7301026C8018230C900A630BE
:1004B0001026C8015030C900A6301026C8016E3081
:1004C000C900F53010263E080D3C031D6B2AC801FB
:1004D000C901003010260230CB0004305826063007
:1004E000DF26CB0110305826C8019430C900A63051
:1004F00010260130C425912A3E080C3C031D8F2A8A
:10050000D8253C0EF0393D07C4000F30C800440820
:10051000C90044081026F6250130C425912A3F3031
:10052000A8000800C70044082C26CB01013058263B
:100530003D08CB00043058263C08CB000430582638
:100540003B08CB00043058263A08CB00023058262E
:10055000CB010130582646082C263F08EE26C70856
:100560000319B42A47082C2645082C2601303726C3
:10057000C80004303726AA0004303726AB00043008
:100580003726AC0002303726AD0001303726C800D0
:100590003E08013C031DD62A3B082C02031DD42A29
:1005A0003A082D020319D62A3F30A8003D082A0236
:1005B000031DDE2A3C082B020319E02A3F30A80065
:1005C00008001030C4002708A8000A303E02031CAF
:1005D000EB2A1230C4004008C500C508031DF12AEB
:1005E0008F2B3E08053C0319012B3E08073C0319DD
:1005F000012B3E08033C0319012B3E08013C031D5F
:100600000E2B043091234008013C0318082BA7232C
:100610000430362704304402C4008D2B3E08043CCD
:1006200003191A2B3E08063C03191A2B3E08023CFC
:10063000031D262B053091233030BA003030BB002B
:100640000430362704304402C4008D2B3E080A3C97
:1006500003192E2B3E080C3C031D412B09300526A7
:10066000C600460E0F396827BC0046080F396827B8
:10067000BD000130C4250230362702304402C400D8
:100680008D2B3E080B3C0319492B3E080D3C031DE6
:100690008B2BC8010E30C90041081026C8016E30EE
:1006A000C900A9301026C8010E30C9004208102622
:1006B000C8016E30C900AA301026C8018030C900B8
:1006C000A6301026C8015030C900A8301026C80135
:1006D0006E30C900F53010263E080D3C031D782B06
:1006E000C801C90100301026C801C9010030102618
:1006F00002300526C600460E0F396827BC004608A2
:100700000F396827BD000130C4250230362702307A
:100710004402C4008D2B3F30A800C503ED2A4408D5
:10072000362FC60046082C2601303726C700043075
:100730003126BD0004303126BC0004303126BB0018
:1007400002303126BA0001303726C70008000A30CF
:100750003E020318B22B2708A80006302C260130D1
:10076000C425B42B3F30A80008002708A800BE010C
:100770000130C0003A0EF0393B07BF00C301C2018F
:10078000C1013D080C3C031D382CBC080319CC2BBF
:100790003C08053C031DD82B0130BE006430C4006A
:1007A000B4263C08053C031DD72B0430C000372C71
:1007B0003C08013C031DE22B0330BE000A30C4009C
:1007C000B426372C3C08023C031DEC2B0530BE0040
:1007D0000A30C400B426372C3C08063C0319F82B19
:1007E0003C08093C0319F82B3C08033C031D172C5B
:1007F0000A30BE000A30C400B4263C08033C031D86
:10080000022CA825C8018E30C900A6301026C801C8
:100810009C30C900A6301026C501C6010030BC2599
:100820003C08063C031D162C0830C000372C3C0841
:10083000043C031D212C0130BE005030C400B426FE
:10084000372C3C08073C0319292C3C08083C031DA5
:10085000352C3C08BE000A30C4003C08083C031D8F
:10086000332C1E30C400B426372C3F30A800A22DF4
:100870003D080D3C031D8F2C2130C200BC0803191C
:10088000452C3C08083C031D4B2C0230BE00643054
:10089000C400B4268E2C3C08013C031D552C0430AA
:1008A000BE006430C400B4268E2C3C08023C031900
:1008B0005D2C3C08073C031D632C0630BE006430F1
:1008C000C400B4268E2C3C08033C03196B2C3C0856
:1008D000093C031D822C0B30BE003C08093C031D63
:1008E000732C0D30BE000A30C400C201B426C8010A
:1008F0009E30C900A6301026C8019C30C900A63021
:1009000010268E2C3C08043C031D8C2C5030C40057
:100910000230BE00B4268E2C3F30A800A22D3D0828
:100920000F3C031DE22C2030C2003C08073C031999
:10093000AC2C3C08083C0319AC2C3C08043C0319C3
:10094000AC2C3C08023C0319AC2C3C08013C0319BC
:10095000AC2CBC08031DC72C0130BE00B4260030EF
:100960002C26C50100301D266430C4003C08023C22
:100970000319BE2C3C08073C031DC02C0530BE00EB
:100980003C08013C031DC62C0330BE00E12C3C0892
:10099000033C0319CF2C3C08093C031DDF2C0C3011
:1009A000BE00B426C8018E30C900A6301026C8018A
:1009B0008C30C900A63010260A30C400E12C3F302C
:1009C000A800A22D3D080E3C031DA02DBC08031D50
:1009D000132DB42600302C263F30C500FF301D26D5
:1009E0000730C50006302C26C50BF22C01302C2612
:1009F00007302C2608302C260A30DF2601302C2622
:100A000007302C26C72603302C26C501FF301D26B3
:100A100008302C260A30DF260B302C2608302C26F6
:100A20000A30DF269F2D3C08013C031D1D2DB426F6
:100A300009302C262830DF269F2D3C08023C031964
:100A4000252D3C08073C031D302DB42600302C26F4
:100A5000C50100301D261F302C260530DF269F2DB6
:100A60003C08043C031D442DB42600302C263F30A6
:100A7000C500FF301D2609302C260A30DF260B303A
:100A80002C260A30DF269F2D3C08083C031D582DDC
:100A9000B42600302C263F30C500FF301D2609301B
:100AA0002C260A30DF260B302C260A30DF269F2D1D
:100AB0003C08033C031D752DB4263C30C500C6011F
:100AC0000430BC250C30C8008030C90080301026AE
:100AD000C801C90100301026CB0104305826063069
:100AE000DF26CB01103058269F2D3C08093C031D02
:100AF0009D2DB4263C30C500C6010530BC250C3008
:100B0000C8000F30C9000F3010263C30C500C601A8
:100B10000430BC250C30C8008730C900873010264F
:100B2000C801C90100301026CB0104305826063018
:100B3000DF26CB01103058269F2D3F30A800A22D74
:100B40003F30A800BF08031DA72D4408BF000800C0
:100B5000C8018E30C900A6301026C8018C30C900EB
:100B6000A63010263C30C500C6010630BC250C302E
:100B7000C800C9010030102EC7004508C300460850
:100B8000C2004708C100D82DC7004708C800C808E0
:100B9000031DCB2DD72D1B27C10AC108031DD52D41
:100BA000C20AC208031DD52DC30AC803C72D0800F9
:100BB000C8010E30C90043081026C8016E30C900B4
:100BC000F8301026C8010E30C90042081026C801AE
:100BD0006E30C900F7301026C8010E30C900410838
:100BE0001026C8016E30C900F630102ECB0103303C
:100BF0005826A512A2272414A6273F08EE26241063
:100C0000A627FD26CB011030582EC7004708CB0081
:100C10000430582608303726C80008303726080028
:100C2000CA004808CB00043058264A08CB000830D8
:100C300058264908CB000830582EC600CB01013099
:100C400058264608CB00083058264508CB00063009
:100C50005826CB010130582EC9004908CB00063078
:100C6000582EC800480837260F3968270800CA00E0
:100C7000A316AF274A08CC00CC08031D402E4E2EE9
:100C80002414A6271B270310CB0CCB13861E492E3A
:100C9000CB172410A6271B27CC033C2EFD264B0880
:100CA000CD004A08083CCE00C727CC004C080800FD
:100CB000CC00A312AF274C08CD00CD08031D612E38
:100CC000702EA5124B1C652EA516A2272414A6274C
:100CD0000310CB0C1B272410A6271B27CD035D2E4A
:100CE000FD2E1A0808009810181D782E4030952601
:100CF00020128C1E7C2E20160800C4008726201E81
:100D0000822E842E1B277E2E440899000800201274
:100D10000C1E8B2E20160800C1271808C427C400FB
:100D20002012C41C942E20160800C400C1272430B1
:100D30009800C4274408C1279900C4279030980020
:100D4000A314B3272311B22FA414A5272214BA2762
:100D5000A316AF27AC26C72EA414A527A01CB32E1C
:100D60002A27C830DF26C72EA01CB92E0A30DF265E
:100D7000BC2E3027C830DF26A414A5272410A627B0
:100D8000A512A2272210BA27A312AF27C72EA51398
:100D9000A027A313AD272517A1272313AE27A4143B
:100DA000A5270130EE26A410A5270130EE26A317B3
:100DB000AD270130EE262317AE270A30EE2EC500F0
:100DC0004508C600C608031DE62EED2E6430C70098
:100DD000FD26C70BE82EC603E22E0800C80048080F
:100DE000C900C908031DF52EFC2E0A30CA00FD26D5
:100DF000CA0BF72EC903F12E08002510201D012F64
:100E00002514A4272019062F2015072F2011A5111E
:100E1000201D0B2FA515A3270000000000000000D7
:100E200000000000000000000000000000000000C2
:100E30000000000008002510201D1F2F2514A427E6
:100E40002019242F2015252F2011A511201D292F11
:100E5000A515A32F2314B427A315B127A0100800AC
:100E60002310B427A311B127A0140800C700470816
:100E7000C800C808031D3D2F672F2A08A9002B08AA
:100E8000AA002C08AB002D08AC002E08AD002F08DE
:100E9000AE003008AF003108B0003208B1003308AE
:100EA000B2003408B3003508B4003608B50037087E
:100EB000B6003808B7003908B8003A08B9003B084E
:100EC000BA003C08BB003D08BC00C803392F08002D
:100ED000C9004908F63E0318073E3A3EC9004908D2
:100EE0000800C4004408BF3E0318F93E113EC40088
:100EF00044080800C40061304402031C852F4408E4
:100F00007A3C031C852FE030C40744080800C50064
:100F10004508C6006430C7000A308E2FC800FF3075
:100F2000C9004708CB004608CA00773049070318B4
:100F3000962FCA0B952FCB0B932FC80B912F080020
:100F4000A72FA72FA72FA72FA72FAA2FAA2F250894
:100F500086000800240885000800BB2FBB2FBB2F8C
:100F6000BB2FBB2FBB2FBB2FBB2FBE2FBE2FBE2F28
:100F7000BE2FBE2FBE2F2308660008002208650082
:100F80000800831603130800831203130800CE0021
:100F90004E08003C031CCD2FD32F0310CD0C013085
:0A0FA0004E02CE00C82F4D080800D5
:02400E00423F2F
:00000001FF
